:100000001529A501A400B7172730A300103014202C
:100010000330A300E8301420A30164301420A301AE
:100020000A30142024081F28A2002508A100240853
:10003000A000F4202008031DB713B71B0800303EB2
:10004000A6003A0884000930A70003102C20A60C53
:10005000A70B262803142C288413B71D3B2800085F
:100060003804371D38068000841700083804031C44
:1000700038068000462800083804031C3806371963
:10008000380680008417380980054628370D063960
:10009000A0004F20A100A00A4F200000BC28003083
:1000A0008A002008820701348B3403342B34003457
:1000B00052340C34EF34A3003A08840038098B2002
:1000C0008413A30803191029F030A50022088038F2
:1000D000A400F030A5030319A5000319A303031915
:1000E00010292008A6002108A7001630BB202608EA
:1000F000A0002708A1009F20030120183808A21F94
:100100003808A20803190301A40F8828800666286E
:10011000892800006928841780051029A000A00DF7
:10012000A00D200D383941389F000030A100323039
:10013000BC201F151F199A28A1011E08102921088B
:1001400020040319A00A8030201AA1062019A10654
:10015000A018A106210DA00DA10D1029A301A20038
:10016000FF30A207031CA307031C10290330A100C2
:10017000E330BC20B028A101F43EA000A109FE306C
:10018000031CC528A0070318C228A0076400A10FFC
:10019000C22800002018CC282018CE280800A10171
:1001A000A301A2000130D928A101A301A2000430BB
:1001B000D928A80023082102031DE02822082002D4
:1001C000043003180130031902302805031DFF30E5
:1001D00010290038031DFF300405031DFF301029CE
:1001E0000404031DFF301029A501A4011030A6004E
:1001F000210DA40DA50D2208A4022308031C230F22
:10020000A50203180A292208A40723080318230FAC
:10021000A5070310A00DA10DA60BF8282008102992
:100220008313031383126400080083161F308500B4
:10023000860170308F008312061083160610831219
:1002400086108316861083120611831606118312F8
:1002500086118316861183120612831606128312E4
:1002600086128316861283120613831606138312D0
:100270008030BE007730BF000130C30040108316CD
:100280009F0106308312BA004030B8006430A200EB
:100290000A305B205A30A20005305B205030A200AB
:1002A00005305B206E30A2000A305B200630BA00B9
:1002B0004030B8006430A20005305B206E30A200F0
:1002C00005305B20061283160612831286168316EB
:1002D0008612831263220630BA004030B8005030D4
:1002E000A20005305B205A30A20005305B20861248
:1002F0008316861283120616831606128312E321D2
:1003000002308E20BC003C08A0006430CF20B20038
:100310003C08A0008230D420B400320884003408A5
:10032000E920B400B5006400340835040319E0295D
:100330000630BA004030B8006430A2000A305B20BA
:100340005A30A20005305B206430A20005305B20EB
:100350006E30A2000A305B205030A20014305B20C7
:100360005A30A20014305B208310401C8314831881
:100370004014831C40100130C20064000630420269
:100380000318C629A3222322C20FBD296400401CE2
:10039000D5290130C2006400063042020318D42976
:1003A000A322E321C20FCB29E0290130C20064005F
:1003B000063042020318E02923226322C20FD72904
:1003C00056296300E129C101061083160610831225
:1003D0008610831686108312861483168610831265
:1003E0000130A3009030AF2043083E02B200B301B9
:1003F000031CB3034108A000A1013308A300320885
:10040000D620B2003E084307B400B501B50D41083F
:10041000A000A1013508A3003408D120B40032089F
:1004200084003408F020B400B500640034083504BA
:1004300003191E2A01308E20C100F429861083166C
:10044000861083120800C10106108316061083125D
:1004500086108316861083120614831606108312E4
:100460000130A3002C30AF2043083F02B200B3019B
:10047000031CB3034108A000A1013308A300320804
:10048000D620B2003F084307B400B501B50D4108BE
:10049000A000A1013508A3003408D120B40032081F
:1004A00084003408F020B400B5006400340835043A
:1004B00003195E2A01308E20C100342A06108316EB
:1004C000061083120800BD0106118316061183125F
:1004D0008611831686118312061583160611831260
:1004E0000130A3009030AF2043083E02B200B301B8
:1004F000031CB3033D08A000A1013308A300320888
:10050000D620B2003E084307B400B501B50D3D0842
:10051000A000A1013508A3003408D120B40032089E
:1005200084003408F020B400B500640034083504B9
:1005300003199E2A00308E20BD00742A06118316EE
:10054000061183120800BD010611831606118312DD
:1005500086118316861183128615831686118312DF
:100560000130A3002C30AF2043083F02B200B3019A
:10057000031CB3033D08A000A1013308A300320807
:10058000D620B2003F084307B400B501B50D3D08C1
:10059000A000A1013508A3003408D120B40032081E
:1005A00084003408F020B400B50064003408350439
:1005B0000319DE2A00308E20BD00B42A861183166E
:1005C00086118312080000308E20BD000630BA006C
:1005D0008030B8000430B700FE302020803020206A
:1005E0004C3020203A3020203D08012020302020AF
:1005F0002030202001308E20C1000630BA0080302B
:10060000B8000430B700FE30202086302020523061
:1006100020203A30202041080120203020202030A6
:10062000202002308E20BC000630BA008030B80096
:100630000430B700FE302020C03020204930202078
:10064000523020203A3020203C0801202030202049
:060650002030202008000C
:02400E00303F41
:00000001FF
